:4000000000080020110000006B0100006B01000010B500F057FE00F05BF900F0AFF8000010B572B69922154B12041A60EE22144B12021A602023C421124A89021360124A57
:40004000124C1160124A18201360D822114B12011A601223236000F0C9FD80220E4B52011A600E4A0E4B1A6000220E4B1A600E4B40321A601123236010BDC0460000024060
:400080000003024000000440080004403000104018000440080304400003014040FF008000000140280003400401014000000000000000000000000000000000000000004B
:4000C0000000000000000000000000000000000000000000000000000000000000000000000000000000000000000000000000000000000000000000000000000000000000
:4001000010B5064C2378002B07D1054B002B02D0044800E000BF0123237010BD1001002000000000FC100000084B10B5002B03D00749084800E000BF07480368002B00D106
:4001400010BD064B002BFBD09847F9E70000000014010020FC100000880000200000000010B562B600F0E0FAFEE710B500F084FF03680C2B00D1FEE7FEE70000F8B50025F0
:400180000F49104B01394A1C14D000221F685C689E68A018B24203D0B858A0500432F8E70200DE68141AA64201D020C2FAE710330139E8E700F066FFFFF7D2FFFEE7C046BC
:4001C0000100000034110000002370B50B480C4C0C4D9A002100032B00D8A95801338150202BF6D1FFF71CFF074B1A68002A00D11A608022054B92051A6070BD00000020EA
:400200006B010000000000008000002008ED00E0004700234118002A05D0013A881800781B18DBB2F7E7180070470000013810B50B2831D8C901494200F00AFF06090B0DAC
:400240000F111513171A1C21FF239B0113E0154B16E0154B0AE0154B12E0154B0BE0154B09E0154B02E0154B00E0154BC91814E0144B05E0144BC9180878C0B211E0134B15
:40028000C9180A7848788C780002230418430300C8781343000603E000210B7848780002184310BDC13F0000C53F0000C93F0000D03F0000D13F0000D63F0000D23F000032
:4002C000D43F0000D83F0000DC3F0000E03F00000C4B10B51A68102313400B4A00D113601368802B0DD10024022021001460FFF79DFFA04205D021000220FFF797FFFFF7F0
:4003000087FF10BD5400034080000020F8B5010006000320FFF78AFF040031000420FFF785FF0134E4012718002431000320FFF77DFF25000130C001B84209D203785A1EE8
:40034000D2B2FD2A00D80125E418E4B20130F3E731000120FFF76AFF6442E4B20623844203D16A4255416D422B401800F8BD0000F0B5BF4CA544019000F00AFA62B6019B8C
:40038000002B02D06B461B7901E0BA4B1B78DBB2039300250A23009502939621039B04AA49000AA800F0FCF9019B002B03D0029B013BDBB20293029B002B02D00028ECD1EC
:4003C00002E0002800D08BE004AB1988062900D849E11A7E0423012A52D104AA568BF21D8A4200D941E1962149008A4200D93CE10AAA92199279172A42D10022F3189BB2CB
:40040000002B09D0A0A99C48C91809180978013B521892B29BB2F3E70AAFBB19597952421B79090292B219430823914228D162E0342B00D0C8E0009B012B00D013E1032EF9
:4004400000D010E18022002155A800F04AFE80251F2155AB581904AB7519F21EC918ADB200F036FE832D00D0F7E004AB9D7F587F2D0205437F2D00D80EE1012300930933E6
:40048000002404AA548001210AAA5370230AD370002311709470221D92B2002A09D0A0A97548891809180978013A5B189BB292B2F3E7A0AA714912195B4251189BB20B7000
:4004C0006F491B0A51180B706E4B0734D2181723137004AAA1B27F3302320AA800F091F9019B002B00D158E7009B012B00D014E10123009351E77B783C79180031380A28E0
:400500002ED9614A1468002C26D0009A012A25D104AAD68007AE13710BAF0C2200213000069700F0DEFDB760310005A8A0472623B488FF339C4202D9B368BB4207D0B2687D
:40054000002A01D1002C04D13368DBB299E70E2396E70E23140094E7052392E705238FE700F080FD0B001900CFFF66FF3800CFFF3C004E0066FF5E006E00009B012B72D19A
:40058000002E70D13000FFF7C1FE43424341009C3B71330075E7009B012B64D1012E62D1002C60D1394B80211B681B689A0BD2B2002A01D19B04590E00237F2239717B719C
:4005C000BA71FB7104245CE7009B012B4BD1022E49D93DE7009B012B45D198E0009B012B41D12C337419FF339C423EDC55AB581932000BA900F06CFD0023A5B21C0040E7EF
:40060000002E30D107AB1900214A350011CA11C10BAA03CB03C2012308240093330030E7009B012B1FD1032E1DD104AA04AB977F5B7F3F021F430A237F2F00D920E748E055
:400640000020FFF763FE002802D18022114B1A6000F0A2F800F046FA05E001230025009302332C000DE704230AE7032308E7C0467CFDFFFF00110000A7FDFFFFACFDFFFFBC
:40068000ADFDFFFFAEFDFFFF2C0100208C0000200411000080000020224B1B681A68D3099BB2520601D001339BB2E0012D18A8B2834204D90123002500930933D1E755A906
:4006C00000F012F90028F5D10123050000930300C7E7E101C919C90180220020FFF799FD0600002C0DD17F2F0BD121000520FFF79DFD2100361A0620FFF798FDF6B2361A3E
:40070000F6B20AAB76421E7101240023B9E60025019BAB4200D0EBE63FE6A1239B009D44F0BDC0468C00002070B50020FFF7EEFD431E98410625144C4042236805401A685C
:40074000C021C03A0020FFF764FD63681B78181AC0B2834203D123681B68002B02D1002000F0BEF9094C2368402B01D0002D03D000202060FFF7FCFD1420FFF7F9FD80234B
:40078000236000F0AFF970BD8C0000208000002010B500F0C1FA10BD10B500F0CBFA10BDF8B504000F0016000120002C28D0002926D00A255D4300F0EBFA002810D000F04B
:4007C000E7FA0500AB2000F06DFA00F0E1FA8542F5D13900AF4200D929003180651807E00120013D00F08AF9002DE4D1102007E0AC4204D000F0B4FA20700134F8E7002069
:40080000F8BD70B501230C001500002805D0002903D000F001FB00232C80180070BD000082B06A460B4B0C4900930C4B01930C4B1A600C4A1160C0461A68120F0F2A04D047
:400840001A680020120F0A2A01D01868C0B202B07047C046B6E9000016000080300100200800104004001040094B0A4A0A491A600A4A1160C0461A68120F0F2A04D01A68AB
:400880000020120F0A2A01D01868C0B27047C04608001040B6E80000150000800400104082B06A460B4B0C4900930C4B01930C4B1A600C4A1160C0461A68120F0F2A04D00B
:4008C0001A680020120F0A2A01D01868C0B202B07047C046B6EA000017000080300100200800104004001040F0B50024A7B00294060003947F2854D8A14252D0802206A820
:4009000000F0E6FB294B04AF04937F23284D7B60284A294B2F601360C0462B6801921B0F0F2B03D02B681B0F0A2B01D02C68E4B20294029B002B36D100F0D7F90400FFF7DF
:400940006FFF0390039B002B02D1FFF78DFF0290029B002B16D1194A19490492049A0198360416430496124A2F600160C0462968090F0F2903D01168090F0A2901D0136842
:40098000DBB20293039B002B07D1FFF789FF0390039B002B01D0039B0293200000F0A9F901E004230293029827B0F0BDB6D70000080010400400104004000080B6D80000DE
:4009C0000500008010B5040000F08FF9102C04D803210C4A13688B430FE0202C05D80321084A13688B43023906E0302C06D80321044A13688B4301390B43136000F079F90C
:400A000010BDC046300010400B480C4A0C4B10B51B68116804680B4A9B00224002601C2213400A07920F1833D340074A9B181B78064ADBB2136010BD00000740280003407B
:400A4000080F0340FFFFFFBFCDF1FF0F0C0F0340024B18684000C00F7047C04600000740024B8000C31818681960704740000020F8B5032605003540B5400F00040006350B
:400A8000AE40AF4000F031F9A408054BA400E4182368B3431F43276000F02BF9F8BDC04600E400E01F2318401E3B8340014A13607047C04600E100E01F2318401E3B8340FE
:400AC000014A13607047C04680E100E01F2318401E3B8340014A13607047C04680E200E001BE7047034A044913689BB20B4313607047C0460CED00E00400FA0570B58025CB
:400B000004002D02064BAC4205D9586800F0E4F8044BE418F6E79868604300F0DDF870BD940000200080FFFFF0B585B000F0C4F8002846D000F0D9F80024234A234B0190D5
:400B40001B681068224A234D14602968224A9B001140A022520311431C2213400207920F1833D3401D4A1E4E53438022D2019B18DB0B013B0B432B60336830200393FFF73A
:400B800021FF8021174AC90513680B4313602A68154B1A40170001201034FFF7AFFFA3053B432B60F02CF6D10120FFF7A7FFFF23084A9B053B431360039B0198336000F08D
:400BC00098F805B0F0BDC04628000340080F03400C0F03400800074000F800C040420F003000104000000740FFFF3FC0F7B50500183D0400182D45D80126234B3700EB401B
:400C00009F433FD100F071F80190FFF721FF0097002802D0FFF7F8FE009607271B4E1C4A33681C49BB4333601B4BE3181B78DBB213601A4A1368BB431360194B0A68E3180C
:400C400018787F239A43034013430B60322000F043F8182C0ED033681C3CA408BB433C401C433460322000F037F83368AD08BB431D433560009B012B01D1FFF755FF019886
:400C800000F037F8F7BDC04611111101080F03400C0F0340180F0340CDF1FF0F100F0340B4F1FF0F10B5034B1B7B584300F014F810BDC04694000020014B1868C00F70470B
:400CC00000000740014A024B1A6070476588EDAC38000340000000000230800803D001300238FCD1C046C0467047EFF3108072B6704780F3108870478021064A10B5136817
:400D000009060B4313600820FFF7CCFE00F006F910BDC0460000094010B5054C2378002B03D100F085F801232370FFF7E5FF10BD4801002010B50820FFF7BEFE00F004F980
:400D4000054A082013685B005B0813600022034B1A60FFF7BBFE10BD00000940880F0940084B094A196813680020994208D013680133412B00D103000449C85C1360C0B207
:400D80007047C046E8010020E40100205C010020044B1868044B1A681B68904200D24130C01A7047E8010020E4010020134B144A30B515681C681900A54208D1114B1C68B9
:400DC0001F232340082B02D00F4B186015E013680133402B00D100230C68A342FCD002210A4CC0B221600A4CE0541360094B1A680A4202D11A680A431A6030BDA0010020FA
:400E0000580100200802094040020940800F0940A4010020880F094070B504004518AC4204D02078FFF7C2FF0134F8E770BD000070B50024072104251E4A1F4B08201A60F8
:400E40001E4B1F4A1C601F4B1A601F4B1F4A13601F4A11601F4A063914601F4A11601F4A13601F4B1C601F4B1D60FFF725FE03210820FFF7FDFD1C490820FFF7F1FD1B4B55
:400E80001C601B4B1C601B4B1C601B4B1C601B4B1D601B4B1C601A681A4B1A801A4B1C601A4B1C601A4B1C701A4B1C601A4B1C6070BDC0460B000002000009404000094043
:400EC00001000A00480009400700008000030940040309401003094044000940000209400402094050000940750F0000880E0940C80E0940480F0940080F0940C80F094075
:400F0000880F094050010020E8010020E40100205401002058010020A0010020064A074B11680B40902109040B431360044B1A88044B1A607047C04600000240FFFF0FFFF9
:400F400050010020880F0940064A074B11680B401360064B1A68E423DB001340044A13807047C04600000240FFFF0FFF880F094050010020254B70B51B68002B00D0984710
:400F8000234B1B685B071CD520241F2021490B680133412B00D100231F4A15681F4AAB4203D113681E4B1C7004E012681D4DD2B2EA540B601C4B1B680342E8D104221B4B10
:400FC0001A601B4B1B689B071FD51F20194C1A4A21681368994210D013680133402B00D100231649164DC95CC9B229601360154B1B680340082BEBD104E00221124A1368D2
:401000008B4313600222114B1A6070BD4C010020CC0F0940E8010020E401002040030940540100205C01002008030940C00F09408C0F094058010020A0010020A4010020DC
:401040004002094008020940880F0940800F094002B4714649084900095C49008E4402BC7047C04603B47146490840004900095E49008E4403BC7047014B18687047C0460F
:40108000080100200E4B70B500251E000D4CE41AA410A54204D0AB00F35898470135F8E700F036F8084B00251E00084CE41AA410A54204D0AB00F35898470135F8E770BD0A
:4010C0001C1100001C1100001C11000024110000002310B59A4203D0CC5CC4540133F9E710BD03008218934202D019700133FAE7704700000012000092000000000000003F
:40110000FF000000A9110319003C010143000000F8B5C046F8BC08BC9E46704729010000C9010000F8B5C046F8BC08BC9E467047010100004811000088000020880000004E
:40114000E00000000000000000000000F4100000F8100000010000000000E02EC05D00001800000000366E010000000000000000000000000000000000000000000000009A
:4011800000000000000000000C1100000000000000000000000000000000000000000000000000000000000000000000000000000000000000000000000000000000000012
:4011C0000000000000000000A80000200000000000000000000000000000000000000000000000000000000000000000000000000000000000000000000000000000000027
:401200000008002011120000BD210000BD21000010B5034B83F3088801F064FB00F0D6FF0008002010B572B69922314B12041A60EE22304B12021A6099222F4B31211A6083
:401240002E4B763A1A602E4A2E4B2F4C1A6020222E4B18201A602E4B183A1A60C0222D4B12011A6082222C4B1A602C4A2C4B1A60D8222C4B12011A6002232B4A13602B4AD0
:4012800011602B4A13601033236001F0C9FA8022B820284B52001A602749284B40011960274908602749196027490A60274A28491A60802252010A602649196026490A60EE
:4012C000264A1A600022264B1A60264B41321A60254B03321A60254B043A1A60244B03321A60244B013A1A601123236010BDC0460000024000030240000402400000044075
:40130000361003000800044030001040180004400001044008010440000204403000C00008020440080304400004044008040440180404400403014041FF00800000014096
:401340001003014044FF00800003014040FF00800C03014043FF00800803014042FF00802800034014010140100101400C010140040101400001014010B5064C2378002B6E
:4013800007D1054B002B02D0044800E000BF0123237010BD20010020000000001C2E0000084B10B5002B03D00749084800E000BF07480368002B00D110BD064B002BFBD0EF
:4013C0009847F9E700000000240100201C2E000088000020000000000022012010B5034B1A60034B187000F023FE10BD3C0100208C00002010B50400022000F093FF1020CD
:40140000604000F08FFF10BD10B500F005FC00F06BFD01F027FC01F07BFA012001F05EFC01F082FA72B610BD002110B50348FF2201714171063001F0E8FC10BD3C010020C0
:40144000002110B50448FA2241718171C171083001F0DBFC10BDC0463C02002010B5012802D1FFF7B9FF08E0FA220020034BD2001A60034B187000F0DBFD10BD3C01002022
:401480008C00002010B50F2802D8FFF7B3FF01E000F048FF10BD000070B50425174C23682B4226D000F0FEFF002822D000F0F4FF0023134A2560D3715379D1180133DBB2D5
:4014C00008725371F92B14D9012000F02BFF162000F028FF0B4CA078FFF7D4FF112000F021FF032000F01EFFA3780133A370FFF7A7FF072001F006F970BDC046C00F08400D
:401500003C0200203C03002070B5012001F0E6FB324CE078012816D16368314A0133636093425AD90023E370636000F0FBFE112000F0F8FE207AFFF7A5FF102000F0F2FE2E
:40154000032000F0EFFE274A136801331360264A934206D9254B1B78012B02D10020FFF77DFF00F083FD00F0C5FB214DEB790133DBB2EB71092B30D96B79002B2BD01B4B64
:401580001B78002B08D1E678002E05D1300000F025FD300000F096FB012000F0C3FE162000F0C0FEA078FFF76DFF102000F0BAFE00266B799E4206DA2B000833F05CFFF7C5
:4015C00061FF0136F5E7032000F0ACFEA3780133A370FFF735FF0023EB7170BD3C030020DB0500003C010020CF0700008C0000203C02002070B506000D001400012000F0AA
:4016000091FE3000FFF73EFF2800FFF73BFF2000FFF738FF032000F085FE70BD70B514220500052978D13F4B5C7A132C41D01AD8112C29D033D8102C6DD1012000F072FE9B
:40164000200000F06FFE2800FFF71CFF200000F069FE0020FFF7CEFE0720FFF7CBFE0220FFF7C8FE4FE0422C2AD006D8142C52D1002000F0B3FC00201FE0502C2FD0602CDA
:4016800049D100F009FB42E0102201001000FFF7B1FFFFF7B9FEFA2001F04AF81CE0224A1278002A02D1FFF797FE30E000221A602DE0012000F092FC012000F003FB26E030
:4016C000102201001000FFF795FFFFF79DFEFA2001F02EF801F008FB01F01EF820E0012000F020FE102000F01DFE2800FFF7CAFE102000F017FE0D4BD878FFF7C3FE0A4B27
:401700001878FFF7BFFE032000F00CFE08E010222900100002E0132229001020FFF76AFF70BDC0463C0100208C0000203C030020F0B5142289B004000A2945D1254B9F7AA2
:40174000587ADA7A3F02103817431E7B597B9A7B032838D801F01AFB02111B2A6B461025DA705E7099701D706A46002393800098019900F0FFFB2A0026E0112002AB5E70D3
:401780009970DA7018709F800298039917E0122504ABDA705E7099701D709F800498059900F0E8FB1022210028000FE0132006AB5E709970DA7018709F800698079900F0FE
:4017C000D9FB102200E0132221001220FFF712FF09B0F0BD3C010020F0B51D4C85B00634E37805000193102B2AD114220A2924D1207900F0E3FA16220700FF281DD060791A
:4018000000F0E6FA17220600FF2816D0A07900F0E9FAFF2803D118222900EC3813E0E379227A1B02134302AA17705670907093800298039900F00CFA019A2900132002E0AF
:40184000132201001000FFF7D5FE05B0F0BDC0463C01002070B51D4B05000633DE78102E02D0112E1FD02AE0052903D014222900100027E000F000FD0400012000F052FD63
:40188000142000F04FFD2800FFF7FCFD013C300000F048FD60426041C0B2FFF7F3FD032000F040FD10E00629E0D11879002802D01922012804D100F0D3FC102200E013227A
:4018C00029001420FFF796FE70BDC0463C01002070B505000E000224FFF7B2FD731E9C4206DA064B0633E05C00F0F4FD0134F5E7290010221520FFF77DFE70BD3C010020DC
:4019000010B50100042802D81122002133E01C4AD079137A103806282BD801F037FA040A0E141A202600002010601800FFF776FE24E01A22190011201EE0002010601800CB
:40194000FFF7F6FE1AE0002010601800FFF744FF14E0002010601800FFF77CFF0EE0002010601800FFF7B4FF08E01A221900162002E0122219001020FFF73CFE10BDC04681
:401980003C01002010B5094A1379911DC8540133DBB21371FF2B08D1032806D0152200211020FFF727FEFFF73FFD10BD3C01002070B504261E4D2B68334234D000F09AFCC8
:4019C000002830D000F090FCC3B2C4B22E60022B13D0032B04D0012B16D1FFF725FD1FE0144D2B79002B1ED02000FFF7CBFF2879FFF786FFFFF718FD15E00E4B1A79002A5E
:401A000011D001225A710EE00A4B1A79002A0AD0002259795A71012902D11020604000E02000FFF7AFFF082000F06CFE70BDC046C00F09403C01002073B5002401254D4E96
:401A4000F570746000F03CFC4B4800F047FC082000F044FE00F00CFD484800F017FD072000F03CFEB470347200F0B6F800F004FA200000F0F5FBFF2000F03CFF280001F04E
:401A80002DF93F4800F06EFF01F0ECF862B6162000F020FD6D2000F01DFD0D2000F01AFD522000F017FD452000F014FD532000F011FD452000F00EFD542000F00BFD5F2089
:401AC00000F008FD2E2000F005FD6B462D4D9C7068789C80000203002A78A87813430004184300F035FA782000F022FE2879EA7800020300687913430004184300F028FA8B
:401B0000642000F015FEE879AA7900020300287A13430004184300F01BFA642000F008FE07256B466A465D70062313700199009800F08EF8962000F0FBFD0199009800F051
:401B400087F8082000F0DEFD00F0FAFB00F0DAFBFFF76AFC280000F0D5FD00F0C9FC00F0A9FCFFF76DFCFFF737FCF46001F0A8F873BDC0463C030020B11900009914000040
:401B800009150000202E000010B5FFF755FFFEE710B5012000F0F6FF0E4C2078002802D100F072FB14E02279002A01D1002003E0237A002B03D1012000F066FB01E09A4257
:401BC000F4D9237A0133DBB2092B00D90023237210BDC0464C03002010B5002000F054FB0B4800F0F5FF0B4C06220021A01C01F00CF90023FF20E36023722370237400F0D2
:401C0000FBFF012000F0BEFF00F07AFF10BDC046911B00004C03002010B5002000F034FB00F0B6FF094C06220021A01C01F0EDF80023E36023722370237400F0EBFF01208C
:401C400000F0A0FF00F05CFF10BDC0464C03002037B50F4C0622A51C009001912800694601F0CAF800F04CFF012000F08BFF0C23A178E2784B439B18064A5B00985A00F026
:401C80004DFF00F071FF0023E3600133237037BD4C0300202A2E000007B500236A466946938005228A70033A0A704B700121044A009851740199D3609374FFF7C9FF07BD89
:401CC0004C03002007B5094B6A46187000236946938005228A700A70054A4B70D3600098013301991374FFF7B3FF07BD8D0000204C03002013B52F4BDA68187C511CD9603D
:401D00001C00002828D0012802D002281CD04FE095294DD900220221DA601974264B18780523012806D169468A808B700B706A4604332EE06846828083700170427000988C
:401D40000199FFF785FF33E09022FF3291422FD90022DA601A742AE05A7C002A1BD00E2926D9997CD8600131C9B299740B2908D90132D2B25A749874062A02D9587418705D
:401D800016E06A460023938005339370637C1370A37C5370D3E71878002802D10023E36006E0D8880028F9D0814201D3DA601A7013BDC0464C0300208D000020FF23072848
:401DC00002D8024B40331B5C18007047AA2E0000FF230B2802D8024B48331B5C18007047AA2E0000FF23052802D8024B54331B5C18007047AA2E000010B5012000F010FE17
:401E00001C4C2378002B01D1002002E0FF2B03D1012000F009FC04E0E278002AF8D09342F2D96378002B01D1002002E0FF2B03D1012000F0EDFB04E0E278002AF8D09342E6
:401E4000F2D9A378002B01D1002002E0FF2B03D1012000F0D1FB04E0E278002AF8D09342F2D9E3780133DBB2FF2B00D10023E37010BDC04660030020F8B50327002000F008
:401E8000D3FB002000F0C4FB002000F0B5FB124C124E3A003100200000F0AEFF3A003100201D00F0A9FF10230D4D3A003100681C2B7000F0A1FF00230A48AB80E370A36002
:401EC000237300F0D1FDFF2000F0E2FD012000F0A7FD00F097FDF8BD60030020042F00008E000020F91D0000F8B50327002000F09BFB002000F08CFB002000F07DFB114C3F
:401F0000114E3A003100200000F076FF3A003100201D00F071FF10230C4D3A003100681C2B7000F069FF0023AB80E370A3606373237300F07BFD012000F072FD00F0B6FD41
:401F4000F8BDC04660030020042F00008E00002007B50322019001A9014800F04DFF07BD600300200022024B1A705A709A7070476003002073B5174C0090267B0191164DA2
:401F8000002E05D0A81D0622694600F035FF1FE006226946280000F02FFF28781038032816D8A66000F0F2FE02040808AE800FE06673FFF7D7FF0BE003222100201D66733C
:401FC00000F01AFFAA78EB78697862702170A37073BDC046600300208E000020F8B50123104E114C377B114D20733373002F0ED106222100A01D00F0FFFE1023601CE91C0B
:402000000322237000F0F8FEA780B76009E01023601CE91C0322237000F0EEFE0023A380B360F8BD600300208E000020042F000010B50D4C00280AD12100A01D062200F00A
:40204000DBFE208AE38900041843618A09E02100A01D062200F0D0FEE08AA38A0004218B1843FFF787FF10BD8E00002070B5504DAB682A7B0133AB602C00002A3ED0012A99
:4020800002D0022A24D091E04A4CA178E278607869702870AA70952B00D887E002230026227B2B730E33AE60601C43492370012A02D10631023201E00322093100F09CFEAF
:4020C000A278E3786178A68029706A70AB706DE0384AD1789078A97090215478FF312C7068708B4262D900231089AB602B73D388000418435189FFF73DFF57E02D4D287800
:402100001038032852D800F041FE02051A290023A36009E0AA88934248D30023627BA3609A4208D101336373AA78EB78697862702170A3703AE06373FFF714FF36E0627BCE
:40214000002A33D1AA88934230D3A3796279A3700123217962702170637327E0627B022A24D8002A08D1A9888B4212D30123A2606373FFF7F7FE0CE0012A0AD1F92B08D956
:40218000022363730023691C02322000A36000F033FE637B022B09D1AB88A268934205D80322211D2000627300F026FE70BDC046600300208E000020042F000010B500F078
:4021C000EFFD03680C2B00D1FEE7FEE7F8B500250F49104B01394A1C14D000221F685C689E68A018B24203D0B858A0500432F8E70200DE68141AA64201D020C2FAE7103371
:402200000139E8E700F0D2FDFFF7BEFCFEE7C04601000000382F0000002370B50B480C4C0C4D9A002100032B00D8A95801338150202BF6D1FEF7F6FF074B1A68002A00D1F5
:402240001A608022054B92051A6070BD00000020BD210000001200008000002008ED00E00223044940000A689A43D2B2034013430B60704700000440024B18688007C00F88
:402280007047C04604000440012304490A689A43D2B2034013430B607047C046000004408021064A10B5136809060B431360082000F014FA00F0B6F810BDC04600000940EF
:4022C00010B5054C2378002B03D100F049F801232370FFF7E5FF10BD70030020014B58607047C04670030020014B18687047C04640030940024B18681F2318407047C0467F
:40230000080309408021054B49021A680A431A601968034A0A401A607047C04604030940FFFFFEFF1F2204490B681340082BFBD0024B18607047C046080209404002094078
:402340008021054B49021A680A431A601968034A0A401A607047C04604020940FFFFFEFF70B5002407210425194A1A4B08201A60194B1A4A1C601A4B1A601A4B1A4A1360DC
:402380001A4A11601A4A063914601A4A11601A4A13601A4B1C601A4B1D6000F0A9F90321082000F081F91749082000F075F9164B1C60164B1C60164B1C60164B1C60164BBF
:4023C0001D60164B1C601A68154B1A8070BDC0460B000002000009404000094001000A004800094007000080000309400403094010030940440009400002094004020940B3
:4024000050000940212D0000880E0940C80E0940480F0940080F0940C80F0940880F094078030020064A074B11680B40902109040B431360044B1A88044B1A607047C046C0
:4024400000000240FFFF0FFF78030020880F09408021064A10B5136809060B431360072000F03CF900F0B6F810BDC0460000084010B5054C2378002B03D100F049F8012388
:402480002370FFF7E5FF10BD7C030020014B58607047C0467C030020014B18687047C04640030840024B18681F2318407047C046080308408021054B49021A680A431A60D3
:4024C0001968034A0A401A607047C04604030840FFFFFEFF1F2204490B681340082BFBD0024B18607047C04608020840400208408021054B49021A680A431A601968034A40
:402500000A401A607047C04604020840FFFFFEFF70B50024072501210426194A194B28001A60194B194A1C60194B1A60194B1A4A13601A4A15601A4A14601A4A11601A4A61
:4025400013601A4B1C601A4B1E6000F0D1F82800032100F0A9F82800164900F09DF8164B1C60164B1C60164B1C60164B1C60164B1E60164B1C601A68154B1A8070BDC046A3
:402580000B000002000008404000084001000A00480008400700008000030840040308401003084044000840000208400402084050000840352D0000880E0840C80E08400D
:4025C000480F0840080F0840C80F0840880F084084030020F021054A13688B4360390B431360034B1A88034B1A6070470004024084030020880F08400223044940000A68D6
:402600009A43D2B2034013430B607047000204407F23044AC00111680B401843C0B210607047C0460002044008230449C0000A689A43D2B2034013430B6070470001044078
:402640000B480C4A0C4B10B51B68116804680B4A9B00224002601C2213400A07920F1833D340074A9B181B78064ADBB2136010BD0000074028000340080F0340FFFFFFBF5C
:40268000CDF1FF0F0C0F0340024B18684000C00F7047C04600000740024B8000C31818681960704740000020F8B5032605003540B5400F0004000635AE40AF4000F029FBD4
:4026C000A408054BA400E4182368B3431F43276000F023FBF8BDC04600E400E01F2318401E3B8340014A13607047C04600E100E01F2318401E3B8340014A13607047C04624
:4027000080E100E01F2318401E3B8340014A13607047C04680E200E0034A044913689BB20B4313607047C0460CED00E00400FA0570B5802504002D02064BAC4205D958684F
:4027400000F0DEFA044BE418F6E79868604300F0D7FA70BDA80000200080FFFFF0B585B000F0BAF8002846D000F0D3FA0024234A234B01901B681068224A234D14602968AF
:40278000224A9B001140A022520311431C2213400207920F1833D3401D4A1E4E53438022D2019B18DB0B013B0B432B6033683020039300F0C9FA8021174AC90513680B4364
:4027C00013602A68154B1A40170001201034FFF7AFFFA3053B432B60F02CF6D10120FFF7A7FFFF23084A9B053B431360039B0198336000F092FA05B0F0BDC046280003408B
:40280000080F03400C0F03400800074000F800C040420F003000104000000740FFFF3FC0F7B50500183D0400182D45D80126234B3700EB409F433FD100F06BFA0190FFF753
:4028400023FF0097002802D0FFF7FAFE009607271B4E1C4A33681C49BB4333601B4BE3181B78DBB213601A4A1368BB431360194B0A68E31818787F239A43034013430B606B
:40288000322000F03DFA182C0ED033681C3CA408BB433C401C433460322000F031FA3368AD08BB431D433560009B012B01D1FFF755FF019800F031FAF7BDC046111111013C
:4028C000080F03400C0F0340180F0340CDF1FF0F100F0340B4F1FF0F014B1868C00F704700000740014A024B1A6070476588EDAC38000340044A1368002BFCDB034B000257
:402900001843014B186070470000014044000080034A1368002BFCDB024A014B1A60704700000140440000408022034B52011A60024A034B1A67704780E100E0BD210000B6
:402940000000002010B5040000F0E3F9C021044AA40113688B431C43146000F0DEF910BD0CE400E010B58024054B64011C60054B18670320FFF7E6FF034B1C6010BDC0464A
:4029800080E100E00000002000E100E08022084B92041A600D22074B1A60074B0C3A1A60064BD632FF321A600022054B1A60704700010640240106403801064014010640B0
:4029C0000801064070B50D000400AC4000F0A1F9024B1C6000F0A1F970BDC0460800064010B5012400F095F9054A13682343136000F093F918212000FFF7E4FF10BDC0467C
:402A00000000064010B5054C2378002B03D1FFF7BDFF01232370FFF7E3FF10BD86030020014B18607047C046300106408022034B12011A60024A034BDA66704780E100E0A2
:402A4000BD2100000000002010B5040000F061F9044AA40713689B009B081C43146000F05CF910BD08E400E010B58024054B24011C60054BD8660320FFF7E6FF034B1C6032
:402A800010BDC04680E100E00000002000E100E0044A1368002BFCDB034B00021843014B186070470000014040000080034A1368002BFCDB024A014B1A607047000001405B
:402AC000400000408022084B92041A600D22074B1A60074B0C3A1A60064A074B1A600022064B1A607047C04680010640A4010640B8010640A70A0000940106408801064072
:402B000010B500F006F90421034A13688B43136000F003F910BDC04600000640014B80B2186070479401064070B50D000400AC4000F0EFF8024B1C6000F0EFF870BDC0465A
:402B40000800064010B5042400F0E3F8054A13682343136000F0E1F818212000FFF7E4FF10BDC0460000064010B5054C2378002B03D1FFF7A7FF01232370FFF7E3FF10BDF0
:402B800087030020014B18607047C046B00106408022034B92011A60024A034B5A67704780E100E0BD2100000000002010B5040000F0AFF8044A054B1168A4030B401C43DD
:402BC000146000F0AAF810BD0CE400E0FF3FFFFF10B58024054BA4011C60054B58670320FFF7E4FF034B1C6010BDC04680E100E00000002000E100E0044A1368002BFCDB87
:402C0000034B00021843014B186070470000014041000080034A1368002BFCDB024A014B1A60704700000140410000408022084B92041A600D22074B1A60074B0C3A1A6005
:402C4000FA22064B92001A600022054B1A607047400106406401064078010640540106404801064010B500F054F80221034A13688B43136000F051F810BDC046000006409E
:402C800070B50D000400AC4000F043F8024B1C6000F043F870BDC0460800064010B5022400F037F8054A13682343136000F035F818212000FFF7E4FF10BDC046000006403D
:402CC00010B5054C2378002B03D1FFF7AFFF01232370FFF7E3FF10BD88030020014B18607047C04670010640402210B5024B1A60FFF712FD10BDC0468000002000000000DB
:402D00000230800803D001300238FCD1C046C0467047EFF3108072B6704780F310887047034B10B51B68002B00D0984710BDC04674030020034B10B51B68002B00D09847AE
:402D400010BDC0468003002010B50400FFF7E1FF102C04D803210C4A13688B430FE0202C05D80321084A13688B43023906E0302C06D80321044A13688B4301390B4313607B
:402D8000FFF7CBFF10BDC0463000104002B4714649084900095C49008E4402BC7047C046014B18687047C0461C0100200E4B70B500251E000D4CE41AA410A54204D0AB0006
:402DC000F35898470135F8E700F0A4F8084B00251E00084CE41AA410A54204D0AB00F35898470135F8E770BD202F0000202F0000202F0000282F0000002310B59A4203D0BF
:402E0000CC5CC4540133F9E710BD03008218934202D019700133FAE77047000000000000FF000000FF000000FF00598F4887B17F8878C671636B5A65AA5F4D5A3A5572502F
:402E4000EC4BAA47A443D83F443CE138B035AD32D52F252D9D2A3928F725D623D321ED1F221E711CD81A5619EA1793164F151C14FB12EB11E910F70F110F380E6C0DAB0C32
:402E8000F50B490BA70A0E0A7E09F5087508FB0788071C07B6065606FB05A50554050705BF047B043A04FE03C4038E035B032B03FD02D202AA0284025F023D021D02FF01F0
:402EC000E201C701AE0195017F0169015501420130011F010F01FF00F100E400D700CB00BF00B500AA00A10098000001020304050607000102030405060708090A0B0001D2
:402F000002030405000000FFFFFF00FF00FF000043000000F8B5C046F8BC08BC9E467047A113000019220000F8B5C046F8BC08BC9E46704779130000482F0000880000201F
:402F40009800000070020000000000000101100000000000100000000000010011FFA500F401100000FF0000010000000000E02EC05D00001800000000366E010000000082
:402F800000000000000000000000000000000000000000000000000000000000102F00000000000000000000000000000000000000000000000000000000000000000000D2
:402FC00000000000000000000000000000000000000000000000000000000000BC0000200000000000000000000000000000000000000000000000000000000000000000F5
:403000000000000000000000000000000000000000000000000000000000000000000000000000000000000000000000000000000000000000000000000000000000000090
:403040000000000000000000000000000000000000000000000000000000000000000000000000000000000000000000000000000000000000000000000000000000000050
:403080000000000000000000000000000000000000000000000000000000000000000000000000000000000000000000000000000000000000000000000000000000000010
:4030C00000000000000000000000000000000000000000000000000000000000000000000000000000000000000000000000000000000000000000000000000000000000D0
:403FC000801112000023000000001E0000000000000000000000000000000000000000000000000000000000000000000000000000000000000000000000000000000000DD
:0200000490303A
:0200000050E2CC
:0200000490402A
:1000000000000000000000000000000000000000F0
:0200000490501A
:0C0000000002190311A900011912628B03
:0200000490600A
:0100000001FE
:00000001FF
